:100000000C94C7010C94E4010C94E4010C94E401F9
:100010000C94E4010C94E4010C94E4010C94E401CC
:100020000C94E4010C94E4010C94E4010C94E401BC
:100030000C94E4010C94E4010C94E4010C94E401AC
:100040000C94E4010C94E4010C94E4010C94E4019C
:100050000C94E4010C94E4010C94E4010C9420024F
:100060000C94E4010C94E4010C94E4010C94E4017C
:100070000C94E4010C94E4010C94E4010C94E4016C
:100080000C94E4010C94E4010C94E4010C94E4015C
:100090000C94E4010C94E4010C94E4010C94E4014C
:1000A0000C94E4010C94E4010C94E4016E616E0084
:1000B000696E6600000000000000005F000000079D
:1000C000000700147F147F14242A7F2A12231308A8
:1000D000646236495522500005030000001C22418D
:1000E000000041221C0014083E081408083E0808BD
:1000F0000050300000080808080800606000002078
:10010000100804023E5149453E00427F40004261D2
:100110005149462141454B311814127F102745455E
:1001200045393C4A49493001710905033649494975
:1001300036064949291E00363600000056360000B2
:10014000081422410014141414140041221408024B
:1001500001510906324979413E7E1111117E7F49D4
:100160004949363E414141227F4141221C7F494954
:1001700049417F090909013E4149497A7F08080838
:100180007F00417F41002040413F017F0814224110
:100190007F404040407F020C027F7F0408107F3E7A
:1001A0004141413E7F090909063E4151215E7F09D7
:1001B000192946464949493101017F01013F404023
:1001C000403F1F2040201F3F4038403F6314081429
:1001D0006307087008076151494543007F414100AA
:1001E00002040810200041417F0004020102044083
:1001F00040404040000102040020545454787F489D
:100200004444383844444420384444487F385454A3
:100210005418087E0901020C5252523E7F08040411
:100220007800447D40002040443D007F1028440079
:1002300000417F40007C041804787C08040478386E
:10024000444444387C14141408081414187C7C08A2
:100250000404084854545420043F4440203C404087
:10026000207C1C2040201C3C4030403C442810286E
:10027000440C5050503C4464544C440008364100F7
:1002800000007F00000041360800100808100878C0
:100290004641467800407A10F35A00A0724E180981
:1002A0000010A5D4E80000E87648170000E40B54DD
:1002B000020000CA9A3B000000E1F50500008096AC
:1002C0009800000040420F000000A08601000000DE
:1002D000102700000000E803000000006400000098
:1002E00000000A00000000000100000000002C7661
:1002F000D888DC674F0823DFC1DFAE59E1B1B7967C
:10030000E5E3E453C63AE651997696E8E6C28426D8
:10031000EB898C9B62ED407C6FFCEFBC9C9F40F2B4
:10032000BAA56FA5F490055A2AF75C936B6CF96730
:100330006DC11BFCE0E40D47FEF520E6B500D0EDF5
:10034000902E0300943577050080841E080000205D
:100350004E0A000000C80C333333330F986E1283FB
:100360001141EF8D2114893BE65516CFFEE6DB18CF
:10037000D1844B381BF77C1D901DA4BBE424203294
:1003800084725E228100C9F124ECA1E53D2711248D
:100390001FBECFEFDAE0DEBFCDBF11E0A0E0B1E0DD
:1003A000E8E3F0E202C005900D92A434B107D9F75A
:1003B00015E0A4E4B1E001C01D92A036B107E1F759
:1003C0000E94A3050C941A100C94000021E030E068
:1003D00002C0220F331F6A95E2F720958223089509
:1003E00090E002C0959587956A95E2F7817008952F
:1003F00010924A0110924B0188E080934D019EE0DB
:1004000090934C0180934F018DE080934E01E0E585
:10041000F1E011821082329682E0E431F807C9F7E8
:1004200082E0809367030895AC0120E001C02F5F54
:10043000FA01E20FF11D80818823C9F7822F089508
:100440001F920F920FB60F9211248F939F9380915A
:100450004501909146010196909346018093450194
:100460009F918F910F900FBE0F901F9018956F92D4
:100470007F928F929F92AF92BF92CF92DF92EF9234
:10048000FF920F931F93DF93CF93CDB7DEB76097A3
:100490000FB6F894DEBF0FBECDBF0E9460098091F9
:1004A000470190914801009751F50EE211E062E199
:1004B000F62E55E0E52ED8012D913C9190E001C03B
:1004C0009F5FF901E90FF11D80818823C9F79E9D87
:1004D000C001112462E070E00E94770DCB0190957D
:1004E00081959F4F865D6F2DA9010E94350BB9E064
:1004F000FB0E0E5F1F4FE4E2FE16E9F606C18130E7
:10050000910509F0E2C08DB79EB708970FB6F89431
:100510009EBF0FBE8DBFEDB7FEB731968E010F5F48
:100520001F4FADB7BEB712961C930E93119780E084
:1005300091E093838283809144018483158280912A
:100540001201992787FD9095978386830E943C0F1F
:10055000EDB7FEB738960FB6F894FEBF0FBEEDBFED
:1005600080E060E0A8010E94350B4CE4C42E41E01D
:10057000D42EAA24BB2433E0632E34C0D6018C9140
:10058000869D702C112411968C91B62D8B02C00182
:10059000112428E0822E880EEE24FF2499E0992E63
:1005A000980E082F065F172D1E0D812F682D41E034
:1005B0000E946809812F692D41E00E946809812FFE
:1005C000602F41E00E9468090894E11CF11CE3E0FF
:1005D000EE16F10441F70894A11CB11C82E090E0F2
:1005E000C80ED91E8091670390E0A816B90634F2B0
:1005F00000E017C080911502A3E08A02C001112417
:10060000609116026A02B0011124685F610F800FC9
:1006100041E00E9468091F5F133061F70F5F0330EC
:1006200011F010E0E7CF80914901813009F06DC0F1
:1006300087E1C82E82E0D82EAA24BB243EC0F60152
:100640002081318182819381892BB1F4F3E02F02E3
:10065000C0011124F82E3F0280011124075F602F92
:1006600041E00E9468098F2D8F5F602F41E00E945A
:1006700068098F2D8E5F16C043E02402700111249B
:10068000E394340280011124602F685F8E2D41E0D5
:100690000E946809602F675F8E2D41E00E94680903
:1006A000065F8E2D602F41E00E9468090894A11C0E
:1006B000B11C84E090E0C80ED91E8091140290E035
:1006C000A816B9060CF4BBCF20C00297F1F4209114
:1006D0003C0130913D0190E001C09F5FF901E90FBD
:1006E000F11D80818823C9F785E0989FC0011124FE
:1006F00062E070E00E94770DCB01909581959F4F4D
:10070000865D62E1A9010E94350B0E945A0B60963A
:100710000FB6F894DEBF0FBECDBFCF91DF911F9112
:100720000F91FF90EF90DF90CF90BF90AF909F9090
:100730008F907F906F9008950E94120E6CE170E090
:100740000E94770D809315020E94120E6DE070E0FA
:100750000E94770D982F8093160280916703482F8F
:1007600050E070911502ECE4F1E020E030E00BC0C5
:100770008081871729F48181891711F461E007C00E
:100780002F5F3F4F32962417350794F360E0809136
:1007900049018130A9F480911402482F50E0E7E12B
:1007A000F2E020E030E009C08081871719F48181F0
:1007B000891711F22F5F3F4F349624173507A4F3A2
:1007C000662309F0B9CF08950F931F9387FF02C0E6
:1007D0000BE105C08C3114F000E001C0082F67FF69
:1007E00002C01CE005C06D3014F010E001C0162FEF
:1007F000809115020817B9F480911602181799F420
:100800009091440180914901813011F081E001C053
:1008100082E0890F809344010E949C0380916703CA
:100820008F5F809367038091670390E00197FC01DD
:10083000EE0FFF1FE45BFE4F20E030E0AC010CC088
:100840009081901719F481818117F9F08181838358
:1008500092832F5F3F4F3297CA01821B930B8F5FAA
:100860009F4F71F7809149018130E9F48091140222
:10087000482F50E0E7E1F2E020E030E011C0808155
:100880009181081751F4191741F480911201815098
:10089000809312010E94F8010AC02F5F3F4F3496E7
:1008A0002417350764F310934D0100934C011F91F9
:1008B0000F910895CF92DF92EF92FF921F93CF9303
:1008C000DF9385E080931201109244010E94F801A9
:1008D000109214020E94120E63E070E00E94770DE5
:1008E00062E0E62EF12CE80EF91EC0E0D0E051E007
:1008F000C52ED12C68C00E94120E62E070E00E94EA
:10090000770D019779F50E94120E6CE170E00E945C
:10091000770D039714F413E007C00E94120E6CE1E8
:1009200070E00E94770D182F0E94120E6DE070E0AB
:100930000E94770D2091140290E00FC0F0E0EE0FBE
:10094000FF1FEE0FFF1FDF01A75EBD4F1D921C9220
:10095000E95EFD4F908381839F5FE92FE20F91173E
:1009600069F72EC00E94120E6DE070E00E94770DB4
:10097000039714F413E007C00E94120E6DE070E0BC
:100980000E94770D182F0E94120E6CE170E00E94F9
:10099000770D2091140290E00FC0F0E0EE0FFF1FE2
:1009A000EE0FFF1FDF01A75EBD4FCD92DC92E95E27
:1009B000FD4F808391839F5FE92FE20F911769F7C5
:1009C000E09314022196CE15DF050CF494CF0E941B
:1009D0009C0381E090E09093480180934701DF9170
:1009E000CF911F91FF90EF90DF90CF90089580916D
:1009F000470190914801009751F4809145019091F1
:100A00004601CD970CF49EC00E945A04089581308F
:100A1000910509F087C020914501309146018091F0
:100A20003E0190E0821793078CF520914A01222322
:100A300021F480914B01882349F190914C01609100
:100A40004B0180914D01680F822F890F0E94E403B2
:100A5000109246011092450180917C00887F816050
:100A600080937C0080917A00806480937A008091EA
:100A70007A0086FDFCCF809178009091790066E63F
:100A800070E00E94630D6E5F60933E0189B18695B0
:100A900080FF04C010924A018FEF1DC083B186957C
:100AA00080FF04C08FEF80934A0107C089B1982F5F
:100AB000917080FF05C090934A0110924B010DC0C8
:100AC00083B190E0880F892F881F990B8170813046
:100AD00021F410924A0180934B018FB18295869543
:100AE000877080FF03C0109249010DC08FB190E064
:100AF00076E0959587957A95E1F7982F917080FF2C
:100B000002C0909349018091120187FF1BC082E0CF
:100B100090E0909348018093470110924601109213
:100B200045010895029771F4809145019091460125
:100B3000CD9744F01092480110924701109246015F
:100B400010924501089580E88093610081E08093D0
:100B500061008FE30E948E0B5998299858982F981E
:100B60008D988E9885B5877F85BD85B5856085BD57
:100B700085B58D7F85BD80916E00816080936E000C
:100B8000789480E480937C0087E880937A0084EFF7
:100B900091E028EC30E0F9013197F1F70197D9F7AE
:100BA00010924601109245010E94F7040E943702FC
:100BB000FBCFA1E1B0E0EFEDF5E00C948A0D3C0134
:100BC0007F876E876A01FC0117821682838181FD0F
:100BD00003C06FEF7FEF6FC39E012F5F3F4F398BD5
:100BE000288BF3012381EE85FF8523FD859123FF6B
:100BF0008191FF87EE87882309F45AC3853251F427
:100C0000EE85FF8523FD859123FF8191FF87EE8788
:100C1000853229F490E0B3010E94100FE2CF982FA3
:100C200010E0882499241032B0F49B3269F09C3291
:100C300028F4903251F0933271F40BC09D3239F0A8
:100C4000903349F4116028C01260146025C0186008
:100C500023C0106121C017FD2AC0892F80538A301C
:100C600078F416FF06C0FAE09F9E902C1124980E8F
:100C700013C03AE0839E802C1124880E10620CC0B1
:100C80009E3221F416FD14C3106406C09C3611F484
:100C9000106802C0983659F4EE85FF8523FD9591C2
:100CA00023FF9191FF87EE87992309F0BCCF892F0D
:100CB0008554833020F4812F8061905E07C0892F96
:100CC0008556833008F09FC1812F8F7E86FD02C03C
:100CD00076E0972E6FE3F62EF822953619F4F0E4BD
:100CE000FF2A07C0963619F420E8F22A02C09110B4
:100CF0009A94F7FE0AC03BE3391518F45CE3B52E6D
:100D000002C0B92CB39427E009C047E0491520F48C
:100D1000BB2447E0942EF7CF292DBB24C6010496AF
:100D20009D878C87F6016081718182819381AE01FC
:100D30004F5F5F4F0B2D0E94220E6C010981202E08
:100D4000332400FF04C003FD02C01DE209C0F1FE10
:100D500002C01BE205C0F2FC02C010E001C010E2BC
:100D6000C1018C709070892BB9F1112311F483E0CB
:100D700001C084E0881510F088240AC0881AF3FCAA
:100D800007C080E290E0B3010E94100F8A94C9F777
:100D9000112329F0812F90E0B3010E94100F23FE50
:100DA00003C00CEA10E00EC000EB10E00BC0E11431
:100DB000F10409F0805290E0B3010E94100F0F5F20
:100DC0001F4F05C0EF2CFF24F0E1EF22FF24F801B4
:100DD0008491882361F714C1F7FE12C0BC0C24FE75
:100DE00004C08A81813309F4BA941B141CF0BB241B
:100DF000B3942DC0F8E0FB1550F538E0B32E27C0B2
:100E0000F6FC25C0892D90E08C159D054CF02CEF4B
:100E1000C2162FEFD20624F030E8F32A01C09A94CC
:100E2000992049F0E2E0F0E0EC0FFD1FE90DF11D23
:100E300080818033A1F3F7FE0AC0B92CB394892DC9
:100E400090E0C816D90614F0992401C09C18F7FC4C
:100E500003C025E030E009C01C141D041CF021E093
:100E600030E003C096012F5F3F4F112311F02F5F39
:100E70003F4F992029F0892D90E00196280F391FC6
:100E8000882D90E02817390714F0882401C0821AB1
:100E90004F2C5524C20189709070892B39F008C0FD
:100EA00080E290E0B3010E94100F8A948820C1F77D
:100EB000112329F0812F90E0B3010E94100F43FE0F
:100EC00007C008C080E390E0B3010E94100F8A942D
:100ED0008820C1F7F7FE46C08601D7FE02C000E0B9
:100EE00010E076010894E11CF11CE01AF10A41E0DF
:100EF00050E04C0F5D1FE40EF51E26014B18510803
:100F0000892D90E0AA24BB24A81AB90A5FEF0F3FED
:100F1000150729F48EE290E0B3010E94100FC0166D
:100F2000D10634F0401651061CF4F701808101C04F
:100F300080E3015010400894E11CF11C0A151B05C8
:100F40002CF090E0B3010E94100FE0CF0C151D05AE
:100F500039F49A81963318F4953311F424FE81E321
:100F600090E04BC08A81813309F00F7E90E0B3019D
:100F70000E94100F9920A1F08EE290E0B3010E9430
:100F8000100F12E0E1E0F0E0EC0FFD1FE10FF11DAA
:100F90001F5F808190E0B3010E94100F9A9491F737
:100FA00044FC03C085E690E002C085E490E0B30114
:100FB0000E94100FD7FC05C0C114D10441F404FFF6
:100FC00006C0D094C194D108D3948DE201C08BE2C5
:100FD00090E0B3010E94100F80E305C08F5F26EF01
:100FE0003FEFC20ED31E3AE0C316D104BCF790E027
:100FF000B3010E94100FC601C096B3010E94100FEA
:10100000CC84DD8452C1933631F0933799F0933517
:1010100009F059C023C0F601808189835E010894DC
:10102000A11CB11C22E030E0C20ED31E21E0E22E52
:10103000F12C12C0F601A080B18016FD03C06FEF45
:101040007FEF02C0692D70E022E030E0C20ED31EB7
:10105000C5010E94050F7C011F7713C0F601A08017
:10106000B18016FD03C06FEF7FEF02C0692D70E005
:1010700022E030E0C20ED31EC5010E94FA0E7C01B0
:10108000106813FF07C01BC080E290E0B3010E940C
:10109000100F8A94882D90E0E816F906A8F30FC087
:1010A000F50117FD859117FF81915F0190E0B30174
:1010B0000E94100F81108A940894E108F108E1144D
:1010C000F10471F7F2C0943611F0993689F517FFE3
:1010D00008C0F601208131814281538184E090E093
:1010E0000AC0F601808191819C01442737FD40951B
:1010F000542F82E090E0C80ED91E9FE6F92EF1220F
:1011000057FF09C050954095309521953F4F4F4F5F
:101110005F4F90E8F92ACA01B901AE014F5F5F4FF6
:101120002AE030E00E94600FE82EE889EE1A41C004
:10113000953721F41F7E2AE030E01CC0197F9F36CE
:1011400061F0903720F4983509F0B2C00FC09037A5
:1011500039F0983709F0ACC004C028E030E00AC08C
:10116000106114FD146020E130E004C014FD16602D
:1011700020E132E017FF08C0F601608171818281B1
:10118000938144E050E008C0F60180819181BC0168
:1011900080E090E042E050E0C40ED51EAE014F5F0B
:1011A0005F4F0E94600FE82E5889E51A8FE7F82EEE
:1011B000F122F6FE0BC08EEFF822E91438F4F4FEAB
:1011C00007C0F2FC05C09FEEF92202C01E2D01C02F
:1011D000192DF4FE0DC0FE01EE0DF11D808180334E
:1011E00019F4E9EEFE2208C01F5FF2FE05C003C03D
:1011F0008F2D867809F01F5F0F2DF3FC14C0F0FED1
:101200000FC0181510F09E2C0BC09E2C980C911A34
:10121000182D06C080E290E0B3010E94100F1F5FFE
:101220001815C0F304C0181510F4811A01C08824E1
:1012300004FF0FC080E390E0B3010E94100F02FF93
:101240001DC001FD03C088E790E00EC088E590E076
:101250000BC0802F867891F001FF02C08BE201C0A5
:1012600080E2F7FC8DE290E0B3010E94100F06C00F
:1012700080E390E0B3010E94100F9A94E914C0F348
:10128000EA94E1E0F0E0EC0FFD1FEE0DF11D80812E
:1012900090E0B3010E94100FEE2091F706C080E2AB
:1012A00090E0B3010E94100F8A948820C1F799CC76
:1012B000F30166817781CB016196E2E10C94A60D82
:1012C000E8E6F3E0119285E0E036F807D9F70895F3
:1012D000843580F5603370F5262F26952695269562
:1012E000677090E0442399F0E4E52E9FF00111240B
:1012F000E80FF91FE859FC4F81E090E002C0880F29
:10130000991F6A95E2F72081282B20830895E4E550
:101310002E9FF0011124E80FF91FE859FC4F81E0DE
:1013200090E002C0880F991F6A95E2F780952081AE
:101330002823208308952F923F924F925F926F92BD
:101340007F928F929F92AF92BF92CF92DF92EF9255
:10135000FF920F931F93DF93CF93CDB7DEB72D97F7
:101360000FB6F894DEBF0FBECDBFD82EC62E142FF9
:10137000022F8417F9F4A62EBB24E22EFF240EC000
:101380008D2D6A2D41E00E946809C01620F4089452
:10139000A11CB11C03C00894A108B108C01628F410
:1013A000EA14FB040CF4FEC0EBCFAE14BF040CF443
:1013B000F9C0E6CF282F30E06017F9F4C9015C01CD
:1013C000E42EFF240EC08A2D6C2D41E00E94680996
:1013D000D11620F40894A11CB11C03C00894A108E4
:1013E000B108D11628F4EA14FB040CF4DBC0EBCFEF
:1013F000AE14BF040CF4D6C0E6CF842F90E09A83DD
:101400008983C9015C0169817A81681B790B88270E
:1014100077FD8095982F0E94AF0C6F83788789871E
:101420009A87202E33244C2C5524B1016419750958
:10143000882777FD8095982F0E94AF0C3B014C01C7
:101440002F81388549855A850E94450C6B837C83A2
:101450008D839E8320E030E040E050E00E945F0DED
:1014600087FF0DC0C401B30190582F81388549858D
:101470005A850E94450C6B837C838D839E830F2E3F
:10148000F0E0CF2EF0E0DF2EF0E0EF2EF0E0FF2EC8
:10149000F02D70C0AB868A2D642D41E00E94680952
:1014A000C701B6012B813C814D815E810E94DD0B1D
:1014B00031C08B85642D41E00E9468091D861C8621
:1014C000C401B30120E030E040E050E00E945F0D35
:1014D000181624F4E1E0F0E0FD87EC8700E010E06E
:1014E000C401B30120E030E040E050E00E94410C34
:1014F000882314F401E010E08C859D85801B910BFE
:10150000480E591EC701B60120E030E040E85FE315
:101510000E94DC0B6B017C0120E030E040E05FE3E7
:101520000E945F0D88239CF0C401B30120E030E0ED
:1015300040E050E00E945F0D18162CF4241435048E
:101540000CF0B7CF04C0421453040CF0B2CF6F813B
:10155000788589859A8520E030E040E050E00E945F
:101560005F0D181624F40894A11CB11C03C0089444
:10157000A108B1086F81788589859A8520E030E0DF
:1015800040E050E00E945F0D181634F4E981FA81C2
:10159000EA15FB053CF07ECF89819A81A816B90631
:1015A0000CF078CF2D960FB6F894DEBF0FBECDBFEE
:1015B000CF91DF911F910F91FF90EF90DF90CF902F
:1015C000BF90AF909F908F907F906F905F904F9063
:1015D0003F902F9008959F92AF92BF92CF92DF924B
:1015E000EF92FF920F931F93CF93DF93982EC62E07
:1015F00085E0489FE0011124C05AD04000E081E01E
:10160000A82EB12C18C0612F6C0DA501012E02C0AF
:10161000440F551F0A94E2F74E215F21012E02C0AC
:10162000559547950A94E2F78D2D0E9468091F5F32
:10163000183049F70F5F053061F0FE01E00FF11D32
:10164000EC54FF4F10E0E491D02ED90CEE2EFF2485
:10165000EFCFDF91CF911F910F91FF90EF90DF902F
:10166000CF90BF90AF909F900895EF92FF920F930D
:101670001F93CF93DF93F82E062F142F242F352F8F
:10168000C901EC0195E0E92E08C08E9DC00111242E
:101690008F0D602F0E94EB0A21969E01211B822F45
:1016A0004881442391F7DF91CF911F910F91FF90D3
:1016B000EF900895CF93DF9380E060E00E94CF0B1E
:1016C000C8E6D3E081E069910E946D0B85E0C036E9
:1016D000D807C1F7DF91CF91089595B18295880F12
:1016E000807E9F7D982B95B95F9827E030E070E071
:1016F0008F98CB01022E02C0959587950A94E2F748
:1017000080FF02C02E9A01C02E988F9A215030403F
:101710008FEF2F3F380761F75F9A08951F93182FB7
:10172000579A249A259A269A879A2C985F9A2C9AE7
:1017300080E061E20E946D0B106880E0612F0E94E2
:101740006D0B80E064E00E946D0B80E063E10E941D
:101750006D0B80E06CE00E946D0B80E060E20E9407
:101760006D0B80E06CE00E946D0B80E060E40E94F5
:101770006D0B80E060E80E946D0B1F910895CF9380
:10178000DF93C0E0D0E081E060E00E946D0B219625
:1017900081E0C83FD807B9F7DF91CF9108951F9333
:1017A000182F606480E00E946D0B106880E0612F4C
:1017B0000E946D0B1F9108955058BB27AA270ED089
:1017C00044C135D130F03AD120F031F49F3F11F4CB
:1017D0001EF42AC10EF4E095E7FB20C1E92F46D1A3
:1017E00080F3BA17620773078407950718F071F43E
:1017F0009EF55EC10EF4E0950B2EBA2FA02D0B01C5
:10180000B90190010C01CA01A0011124FF27591B45
:1018100099F0593F50F4503E68F11A16F040A22F4B
:10182000232F342F4427585FF3CF469537952795BC
:10183000A795F0405395C9F77EF41F16BA0B620BBB
:10184000730B840BBAF09150A1F0FF0FBB1F661F02
:10185000771F881FC2F70EC0BA0F621F731F841F45
:1018600048F4879577956795B795F7959E3F08F06B
:10187000B3CF9395880F08F09927EE0F979587952A
:101880000895A8D008F481E008950CD0DEC0D6D029
:1018900040F0CDD030F021F45F3F19F0BFC05111BE
:1018A00008C1C2C0E3D098F39923C9F35523B1F31B
:1018B000951B550BBB27AA2762177307840738F0BF
:1018C0009F5F5F4F220F331F441FAA1FA9F333D01E
:1018D0000E2E3AF0E0E830D091505040E695001CD2
:1018E000CAF729D0FE2F27D0660F771F881FBB1F8E
:1018F000261737074807AB07B0E809F0BB0B802D68
:10190000BF01FF2793585F4F2AF09E3F510568F0B3
:1019100085C0CFC05F3FECF3983EDCF386957795AA
:101920006795B795F7959F5FC9F7880F911D9695B5
:10193000879597F90895E1E0660F771F881FBB1F11
:10194000621773078407BA0720F0621B730B840BBE
:10195000BA0BEE1F88F7E0950895E89409C097FB4D
:101960003EF490958095709561957F4F8F4F9F4F76
:101970009923A9F0F92F96E9BB279395F6958795BA
:1019800077956795B795F111F8CFFAF4BB0F11F47D
:1019900060FF1BC06F5F7F4F8F4F9F4F16C0882324
:1019A00011F096E911C0772321F09EE8872F762F5A
:1019B00005C0662371F096E8862F70E060E02AF09B
:1019C0009A95660F771F881FDAF7880F9695879587
:1019D00097F90895990F0008550FAA0BE0E8FEEF5C
:1019E00016161706E807F907C0F012161306E407E3
:1019F000F50798F0621B730B840B950B39F40A26DC
:101A000061F0232B242B252B21F408950A2609F4B9
:101A1000A140A6958FEF811D811D089597F99F67BD
:101A200080E870E060E008959FEF80EC0895002466
:101A30000A941616170618060906089500240A9433
:101A400012161306140605060895092E0394000CB9
:101A500011F4882352F0BB0F40F4BF2B11F460FF48
:101A600004C06F5F7F4F8F4F9F4F089557FD905871
:101A7000440F551F59F05F3F71F04795880F97FB52
:101A8000991F61F09F3F79F087950895121613060C
:101A90001406551FF2CF4695F1DF08C0161617063B
:101AA0001806991FF1CF8695710561050894089570
:101AB000E894BB2766277727CB0197F908958ADF3B
:101AC00008F48FEF0895AA1BBB1B51E107C0AA1FA2
:101AD000BB1FA617B70710F0A61BB70B881F991FCF
:101AE0005A95A9F780959095BC01CD01089597FB73
:101AF000092E07260AD077FD04D0E5DF06D00020A6
:101B00001AF4709561957F4F0895F6F79095819539
:101B10009F4F08952F923F924F925F926F927F92C4
:101B20008F929F92AF92BF92CF92DF92EF92FF92ED
:101B30000F931F93CF93DF93CDB7DEB7CA1BDB0B99
:101B40000FB6F894DEBF0FBECDBF09942A8839883E
:101B500048885F846E847D848C849B84AA84B98445
:101B6000C884DF80EE80FD800C811B81AA81B98151
:101B7000CE0FD11D0FB6F894DEBF0FBECDBFED0165
:101B80000895A0E0B0E0E7ECFDE00C94920DEC01CC
:101B9000A880B980CA80DB80A114B104C104D1043B
:101BA00041F484E2A82E89EDB82E8BE5C82E87E09B
:101BB000D82EC601B5012DE133EF41E050E00E947F
:101BC000DD0F27EA31E440E050E00E94BE0F7B01C8
:101BD0008C01C601B5012DE133EF41E050E00E94D8
:101BE000DD0FCA01B9012CEE34EF4FEF5FEF0E9419
:101BF000BE0F6E0D7F1D801F911F97FF04C06150A7
:101C0000704080409048688379838A839B839B01DE
:101C10003F77C901CDB7DEB7EAE00C94AE0D0E9464
:101C2000C10D08958FE391E00E94C10D0895A0E0D9
:101C3000B0E080933F0190934001A0934101B093A5
:101C400042010895283008F027E03327DA01990F80
:101C5000311D87FD916000966105710539F4326090
:101C60002E5F3D9330E32A95E1F708959F3F30F0D2
:101C700080387105610509F03C5F3C5F3D93913010
:101C800008F08068911DDF93CF931F930F93FF920D
:101C9000EF92192F987F9695E92F96959695E90FD3
:101CA000FF27E251FD4F99273327EE24FF24A70198
:101CB000E70105900894079428F4360FE71EF81EF4
:101CC000491F511D660F771F881F991F0694A1F7A2
:101CD0000590079428F4E70EF81E491F561FC11DF2
:101CE000770F881F991F661F0694A1F70590079428
:101CF00028F4F80E491F561FC71FD11D880F991FC2
:101D0000661F771F0694A1F70590079420F4490FEA
:101D1000561FC71FD81F990F661F771F881F06946D
:101D2000A9F784911095177041F0D695C7955795EE
:101D30004795F794E7941A95C1F7E4E9F2E06894BF
:101D40001590159135916591959105907FE2739568
:101D5000E118F10A430B560BC90BD009C0F7E10C8F
:101D6000F11E431F561FC91FD01D7EF4703311F49E
:101D70008A95E6CFE894015030F0080F0AF4002766
:101D8000021708F4202F2395022F7A3328F079E3E5
:101D90007D932A95E9F710C07D932A9589F60694DC
:101DA00097956795379517951794E118F10A430BA6
:101DB000560BC90BD00998F023957E9173957A3311
:101DC00008F070E37C932013B8F77E9170617D93E7
:101DD00030F0839571E37D9370E32A95E1F7112448
:101DE000EF90FF900F911F91CF91DF91992787FD81
:101DF00090950895FC010590615070400110D8F74E
:101E0000809590958E0F9F1F0895FC016150704042
:101E100001900110D8F7809590958E0F9F1F08951F
:101E20000F931F93CF93DF938C01EB018B8181FF85
:101E30001BC082FF0DC02E813F818C819D812817A0
:101E4000390764F4E881F9810193F983E88306C0D6
:101E5000E885F985802F0995892B31F48E819F8142
:101E600001969F838E8302C00FEF1FEFC801DF91A1
:101E7000CF911F910F910895AEE0B0E0E2E4FFE052
:101E80000C94980D0D891E8986E08C831A83098332
:101E90008FEF9FE79E838D839E01275E3F4FCE018C
:101EA00001966F89788DA9010E94D9052F81388507
:101EB000020F131FF80110822E96E4E00C94B40D6B
:101EC000FA01AA27283051F1203181F1E8946F936B
:101ED0006E7F6E5F7F4F8F4F9F4FAF4FB1E03ED011
:101EE000B4E03CD0670F781F891F9A1FA11D680FAF
:101EF000791F8A1F911DA11D6A0F711D811D911DE2
:101F0000A11D20D009F468943F912AE0269F112456
:101F10003019305D3193DEF6CF010895462F4770BA
:101F2000405D4193B3E00FD0C9F7F6CF462F4F7015
:101F3000405D4A3318F0495D31FD4052419302D073
:101F4000A9F7EACFB4E0A695979587957795679519
:101F5000BA95C9F700976105710508959B01AC0119
:101F60000A2E06945795479537952795BA95C9F740
:101F7000620F731F841F951FA01D0895629FD001DB
:101F8000739FF001829FE00DF11D649FE00DF11D34
:101F9000929FF00D839FF00D749FF00D659FF00DE3
:101FA0009927729FB00DE11DF91F639FB00DE11DD0
:101FB000F91FBD01CF011124089597FB092E0526B5
:101FC0000ED057FD04D014D00AD0001C38F4509520
:101FD0004095309521953F4F4F4F5F4F0895F6F74D
:101FE00090958095709561957F4F8F4F9F4F089585
:101FF000A1E21A2EAA1BBB1BFD010DC0AA1FBB1F0D
:10200000EE1FFF1FA217B307E407F50720F0A21B7E
:10201000B30BE40BF50B661F771F881F991F1A94EB
:1020200069F760957095809590959B01AC01BD0115
:08203000CF010895F894FFCFE1
:1020380053636F72653A2564204C697665733A2557
:102048006400054279204D617474686577204D6994
:102058006C6C6572006E39333432343031001301E0
:10206800250147616D65204F7665720032010601D2
:042078000000000064
:00000001FF
